:100000000C941E060C9451280C947E280C944606E1
:100010000C9446060C9446060C9446060C94460630
:100020000C9446060C9446060C942C130C9446062D
:100030000C9446060C9446060C9446060C94460610
:100040000C94AB280C9446060C94992C0C94DC2C44
:100050000C9446060C9446060C9446060C944606F0
:100060000C9446060C944606DC183E191D192019FE
:100070002319261929192C192F193E193819701A04
:10008000721A721A701A721A721A721A721A721A12
:10009000721A721A721A721A721A721A721A721A00
:1000A000F619721A721A721A721A721A6719721A79
:1000B000721A721A721A721A721A721A721A721AE0
:1000C000721A721A721A721A721A721A021A021AB0
:1000D000021A021A021A021A021A021A021A721AD0
:1000E000721A721A721A721A721A6719011A011A9E
:1000F000011A011A721A0F1A151A1B1A211A271A35
:100100002D1A331A391A431A4D1A571A611AA81997
:100110006A19721A721A721A721AF619721A721A05
:10012000721A721A721A721A721A721A001A001A53
:10013000001A001A721A0F1A151A1B1A211A271AF6
:100140002D1A331A391A431A4D1A571A611AA81957
:100150006A19721A721A721A721AF619A51AA51A5F
:10016000A51AA51AA51AA51AA51AA51AA51AA51A97
:10017000A51AA51AA51ABC1BBC1BBC1BBC1BBC1B0F
:10018000BC1BEA1AF41AFE1A081B661B701B7F1BA5
:10019000901B181D2D1D391D421D511D761D7F1DE3
:1001A000C81D911DDC20E220E820EF20FD201F214A
:1001B0003D21456E746572206D656E752E2E2E0084
:1001C000546F67676C6564206D6963726F50504D42
:1001D00000546F67676C656420696E76657274653C
:1001E000642050504D2100546F67676C6564205443
:1001F00058206D7574696E672100546F67676C6570
:10020000642074656C656D65747279210050726F3D
:10021000746F636F6C206572726F72207769746897
:100220002052580054696D656F7574207768656E4B
:1002300020636F6E6E656374696E6720746F205201
:100240005800507265737320616E79206B65792058
:10025000746F2063616E63656C00436F6E6E6563DF
:1002600074696E6720746F2052582C20706F776508
:100270007220757020746865205258202877697440
:10028000682062696E6420706C7567206966206EF4
:100290006F74207573696E6720616C776179732064
:1002A00062696E642900546F67676C656420276912
:1002B0006D6D656469617465206F75747075742700
:1002C00000546F67676C65642027736C61766520E6
:1002D0006D6F64652700546F67676C6564202761E4
:1002E0006C776179732062696E642700546F676769
:1002F0006C65642050504D206368616E6E656C20A3
:100300006C696D69740053657420525353492069B8
:100310006E6A656374696F6E206368616E6E656C8A
:100320002028303D3D64697361626C652900536526
:10033000742050504D206D696E696D756D20737914
:100340006E630053657420626561636F6E20696E31
:1003500074657276616C0053657420626561636FC9
:100360006E2064656C617900536574206265616319
:100370006F6E206672657175656E637920696E2097
:10038000487A3A20303D64697361626C652C205074
:10039000783D504D52206368616E6E656C20782CFC
:1003A0002046783D465253206368616E6E656C202E
:1003B00078005365742050574D2073746F7020641B
:1003C000656C61792028302064697361626C6564B2
:1003D0002C20312D323535203D3D20302E317320FB
:1003E0002D2035306D696E29005365742050504DB5
:1003F0002073746F702064656C61792028302064EC
:10040000697361626C65642C20312D323535203D75
:100410003D20302E3173202D2035306D696E29003E
:10042000536574206661696C736166652064656CF0
:1004300061792028302064697361626C65642C20C6
:10044000312D323535203D3D20302E3173202D2089
:1004500035306D696E29002A2A2A2A2A2A2A2A2A50
:100460002A2A2A2A2A2A2A2A2A2A2A2A2A2A2A2AEC
:100470002A2A2A2A0052582041636B6564202D20C5
:1004800072657665727420737563636573736675E0
:100490006C21002A2A2A2A2A2A2A2A2A2A2A2A2AAD
:1004A0002A2A2A2A2A2A2A2A2A2A2A2A2A2A2A2AAC
:1004B000002A2A2A2A2A2A2A2A2A2A2A2A2A2A2AC6
:1004C0002A2A2A2A2A2A2A2A2A2A2A2A2A2A00528E
:1004D000582041636B6564202D20757064617465DC
:1004E000207375636365737366756C21002A2A2A0D
:1004F0002A2A2A2A2A2A2A2A2A2A2A2A2A2A2A2A5C
:100500002A2A2A2A2A2A2A2A2A2A0056616C696457
:100510002063686F69636573206172653A205B319F
:100520005D2D5B31365D20286368616E6E656C20E1
:10053000312D31362900536574206F7574707574D0
:1005400020666F7220706F727420005B585D2061AE
:10055000626F7274206368616E67657320616E6498
:10056000206578697420525820636F6E6669670051
:100570005B535D20736176652073657474696E6783
:100580007320746F205258005B525D20726576654F
:1005900072742052582073657474696E6773207486
:1005A0006F2064656661756C747300557365206EA9
:1005B000756D62657273205B312D445D20746F2010
:1005C0006564697420706F727473205B452D515D92
:1005D00020666F722073657474696E677300202DD6
:1005E00020726563656976657220636F6E66696700
:1005F000757261746F722C20727820737720000AF4
:100600000A6F70656E4C52536E67200053657420FC
:1006100073657269616C2062617564726174653AB8
:10062000200056616C69642063686F696365733A82
:100630002031202D20342B34202F2032202D203823
:10064000202F2033202D20382B34202F2034202D14
:10065000203132202F2035202D2031322B34202FF5
:100660002036202D20313600536574204368616E9A
:100670006E656C20636F6E6669673A20005365741F
:100680002044617461726174652028302D32293AEA
:10069000200053657420486F70206368616E6E653A
:1006A0006C7320286D61782032342C207365706162
:1006B000726174656420627920636F6D6D61732966
:1006C0002076616C69642076616C75657320312DCC
:1006D0003235353A2000536574206368616E6E656B
:1006E0006C2073706163696E6720287831306B48C5
:1006F0007A293A200053657420524620706F77653E
:10070000722028302D37293A200053657420524634
:10071000206D6167696320286865782920652E67E8
:100720002E20307844454144463030443A2000532E
:1007300065742062617365206672657175656E63AC
:10074000792028696E20487A293A20005B5A5D207A
:10075000656E746572207265636569766572206383
:100760006F6E66696775726174696F6E2075746902
:100770006C79005B465D20646973706C61792061FF
:10078000637475616C206672657175656E63696509
:10079000732075736564005B525D2063616C6375E3
:1007A0006C6174652072616E646F6D206B65792079
:1007B000616E6420686F70206C697374005B495DC2
:1007C000207265696E697469616C697A6520736508
:1007D0007474696E677320746F20736B65746368DB
:1007E0002064656661756C7473005B585D2072658A
:1007F00076657274206368616E67657320616E64EC
:100800002065786974206D656E75005B535D20739B
:100810006176652073657474696E677320746F20E8
:10082000454550524F4D20616E64206578697420B3
:100830006D656E7500557365206E756D62657273BA
:10084000205B302D395D20746F20656469742070E1
:100850006172616D657465727300202D2053797328
:1008600074656D20636F6E66696775726174696F18
:100870006E000A0A6F70656E4C52536E672000510D
:1008800029204F7574707574206265666F726520DB
:100890006C696E6B20283D465329203A2000502970
:1008A00020536C617665206D6F64652028657870D3
:1008B0006572696D656E74616C293A20004F29205C
:1008C00054696D65642042494E44206174207374FC
:1008D000617274757020203A20004E292050504DCE
:1008E000206F7574707574206C696D69746564200F
:1008F000202020203A200044495341424C454400E6
:100900004D292050504D205253534920746F20637D
:1009100068616E6E656C202020203A20004C2920F2
:1009200050504D206D696E696D756D2073796E63E1
:10093000202875732920203A200044495341424C15
:100940004544004B29204661696C736166652062ED
:100950006561636F6E20696E74762E2028312D32AA
:10096000353573293A20004A29204661696C736144
:10097000666520626561636F6E2064656C617920D5
:1009800028302D323535203D3E20313073202D204A
:100990003135306D696E293A200049292046616958
:1009A0006C7361666520626561636F6E206672714B
:1009B0002E203A200048292050574D2073746F7024
:1009C0002064656C6179202020202020203A2000BE
:1009D00047292050504D2073746F702064656C61FE
:1009E00079202020202020203A200046292046611E
:1009F000696C736166652064656C617920202020D4
:100A00002020203A200050574D206368616E6E65AB
:100A10006C200066756E6374696F6E3A2000292041
:100A2000706F72742000506F776572546F776572C3
:100A300000445446205548462033322D62697420C4
:100A400031306368004F70656E4C52536E67525878
:100A5000206D696E6920342F36636800466C7974A6
:100A6000726F6E2F4F72616E6765525820554846FF
:100A70002038636800525820747970653A20004429
:100A8000697361626C656400487A00203D3D200016
:100A900043616C63756C61746564207061636B6540
:100AA0007420696E74657276616C3A200042292068
:100AB0004D6963726F202868616C66292050504D23
:100AC000202020203A00412920496E766572746505
:100AD000642050504D20696E20202020203A0030A4
:100AE00029204D7574652062757A7A657220286DAB
:100AF0006F73746C79293A003929205365726961E2
:100B00006C2062617564726174653A00736D617224
:100B100074506F7274004672536B79005472616E38
:100B200073706172656E740044697361626C6564B0
:100B30000038292054656C656D657472793A2020FF
:100B40002020202020003729204368616E6E656CCC
:100B500020636F6E6669673A202000362920446161
:100B60007461726174652028302D32293A2020206A
:100B700000352920486F70206368616E6E656C7364
:100B80003A2020202020003429204368616E6E65C1
:100B90006C2073706163696E673A202000332920EE
:100BA000524620706F7765722028302D37293A2001
:100BB0002020003229205246206D616769633A2067
:100BC0002020202020202020003129204261736530
:100BD000206672657175656E63793A202020000089
:100BE00000000700020100000304060000000000EE
:100BF00000000001020408102040800102040810D7
:100C00002001020408102004040404040404040263
:100C10000202020202030303030303000000002395
:100C2000002600290000000000250028002B0000FD
:100C3000000000240027002A0000CA2D11241FBE36
:100C4000CFEFD8E0DEBFCDBF13E0A0E0B1E0E2EA35
:100C5000F1E602C005900D92A83CB107D9F716E065
:100C6000A8ECB3E001C01D92A239B107E1F71CE086
:100C7000CCE3DCE004C02297FE010E94D32ECA33ED
:100C8000D107C9F70E94062E0C94CF300C940000B7
:100C900080917705813019F482E080937705809107
:100CA0007705833019F484E0809377050895A8953B
:100CB0000895DC01ED91FC910190F081E02D099502
:100CC00008952091780530917905382748E0C901C9
:100CD000880F991F37FF06C09C0151E2252750E17C
:100CE000352701C09C01415091F73093790520933D
:100CF0007805089588E380937A0580E092ECA1E07E
:100D0000B0E080937B0590937C05A0937D05B09324
:100D10007E0587E08093870580EC92E9ADEEB9E12E
:100D200080937F0590938005A0938105B093820501
:100D300085E0809388058DEE9EEFADEABEED809351
:100D4000830590938405A0938505B0938605E9E813
:100D5000F5E080E090E0863028F4DC01AE54BC4F32
:100D60002C9101C020E0219301968831910599F7DB
:100D700082E08093A1058AE08093A205089580EC2B
:100D800091EDA8E9BBE18093BF059093C005A093C6
:100D9000C105B093C20580E090E0A0E0B0E580938B
:100DA000C3059093C405A093C505B093C605E7ECB1
:100DB000F5E080E081938F5F8031E1F70895A0E056
:100DC000B0E0E5EEF6E00C949C2ED82F0E940129AD
:100DD0006115710581059105C9F30E943F2F10929D
:100DE0008305109284051092850510928605C4E053
:100DF000812C912C54018A94C0908305D090840555
:100E0000E0908505F0908605FE2CED2CDC2CCC24A2
:100E10000E943A2FA50194010E947B2E6C0D7D1D2E
:100E20008E1D9F1D609383057093840580938505B7
:100E300090938605C15001F7DD2309F450C009E8FD
:100E400015E0E801A12CB12C62E3C62ED12CE12CD7
:100E5000F12C8881882309F442C0B39419F40E94CC
:100E60007A063DC00E943A2FA70196010E947B2E70
:100E7000E1E0E60FA9E8B5E08A2F801B8A1520F48F
:100E80008D918E13F9CFE9CF2091880530E0A0E154
:100E9000B7E20E94132E9B01AC01AE2FB0E00E947E
:100EA000222E40907F0550908005609081057090C3
:100EB0008205640D751D861D971D4090BF055090DD
:100EC000C0056090C1057090C205461657066806B9
:100ED000790618F2E993A39488E1A812BACFCDB7A6
:100EE000DEB7E0E10C94B82E8436910520F4BC0105
:100EF00080E090E017C09C018E3B910528F42A55B4
:100F00003109AAE0B0E00CC0823D910528F4245BD1
:100F10003109A4E6B0E004C02D5C3109A8E5B2E0D7
:100F20000E94132EA4E6B0E09B01AC010E94222E89
:100F3000089590E08C599F4F0E947407089561E0D6
:100F400083E10E94AE2960E083E10E94E72982E00C
:100F50008093B00085E08093B10061E083E00E945F
:100F6000AE2960E083E00E94E7290895A4E0B0E0A4
:100F7000ECEBF7E00C94AA2E009749F19C0140E0BD
:100F800050E068E478EE81E090E00E947B2E61E022
:100F900083E129833A834B835C830E94E72929817B
:100FA000822F3A81932F4B81A42F5C81B52F8F3FE5
:100FB0009105A105B10529F020F08FEF90E0A0E0A8
:100FC000B0E08093B3008091B000806107C060E022
:100FD00083E10E94E7298091B0008F7E8093B0006A
:100FE0002496E2E00C94C62E60E08CE00E94AE29CC
:100FF00061E08BE00E94AE2961E08DE00E94AE29A5
:1010000060E082E00E94AE2961E084E00E94AE29A7
:10101000089542E050E068E476E080E00E943128E4
:101020000895E3E0F0E089E080935700E491E670F2
:1010300081E0E63009F080E00895CF93DF93C82F78
:101040000E941108882381F0DFB781E08093760544
:10105000F8940E94570688E180936000C093600076
:10106000C1110E945706DFBFDF91CF9108958F9283
:101070009F92AF92BF92CF92DF92EF92FF92CF9367
:10108000FC01C0A5EC2FE770F0E0E658FC4FA08112
:10109000B0E0C7FF03C024E130E002C02FE030E041
:1010A000FC0197A183E1989FF0011124E25CFE4FBF
:1010B00080809180A280B380A20FB31F20E43FE123
:1010C0004DE750E00E942D2EA50194010E94592E5B
:1010D0008C2F887149F469017A01E0EDCE0EE7E0CA
:1010E000DE1EE11CF11C1BC0C7FF05C060E47AE8EE
:1010F0008CE29EE004C060E07EEE8AEB9BE069013A
:101100007A01F8EBCF0EFBE0DF1EE11CF11CA5011C
:1011100094010E94592EC20ED31EE41EF51EC70173
:10112000B60169517C4F8F4F9F4F28EE33E040E06E
:1011300050E00E94592EA8EEB3E00E94222ECF91DB
:10114000FF90EF90DF90CF90BF90AF909F908F90E7
:1011500008958F3F910551F048F0811522E09207E4
:1011600038F08115934030F482E0089580E00895CE
:1011700081E0089583E00895A0E0B0E0E2ECF8E0BB
:101180000C94A52EEB018A01B82FB695A0E028811A
:101190003981F80120832A813B8121832C813D8183
:1011A00022832E813F812383688179814A815B81FB
:1011B0002C813D81EE81FF819F2F9295990F990F90
:1011C000907C272F2370922B252F2370220F220F24
:1011D000922B232F23702295207F922BF80194834A
:1011E0000B5F1F4F2896AF5FBA1788F680FF24C0A9
:1011F000888199810E94A908D82E8A819B810E94AA
:10120000A908E82E8C819D810E94A908F82E8E8164
:101210009F810E94A908F0E4DF9EA001112490E1C3
:10122000E99E90011124242B282BE4E0FE9EB001BE
:101230001124262BF8012083CDB7DEB7E7E00C940C
:10124000C12E803223E0920708F1883E23E0920706
:1012500040F48F519340E4E096958795EA95E1F745
:101260000895803D27E0920718F48C5D934008951F
:10127000883928E0920768F4885C974074E0969576
:1012800087957A95E1F78D509C4F089580E090E026
:1012900008958FEF93E008958C30910540F4A4E019
:1012A000880F991FAA95E1F7885D9C4F0895843FA8
:1012B00023E0920718F484529C4F0895811524E08E
:1012C000920740F48657934FF4E0880F991FFA95E0
:1012D000E1F7089580E998E008959C0136952795F7
:1012E00025753575821B930B9C012373337396957B
:1012F00087959695879583739373820F931F9C01AF
:1013000054E0369527955A95E1F7280F391F2F702D
:101310003F7041E051E0249FC001259F900D349F14
:10132000900D1124892F08952D98882319F000001D
:101330002B9A02C000002B9800002D9A00000895FF
:101340002D9A000083B12D98000082958170089538
:10135000CF93DF93D82F5C9A2D985C98C8E08D2F9F
:1013600080780E949409DD0FC150C9F72D98DF9154
:10137000CF9108958F770E94A8090895CF93DF93A6
:10138000D82FC8E08D2F80780E949409DD0FC150BE
:10139000C9F72D98DF91CF910895CF93DF932D98C2
:1013A000C8E080E0D82FDD0F0E94A0098D0FC1504A
:1013B000C9F7DF91CF9108950E94BA090E94CD0923
:1013C0005C9A0895A1E0B0E0E8EEF9E00C94AA2E52
:1013D000806869830E94A8096981862F0E94BE09DE
:1013E0005C9A2196E2E00C94C62ECF93C0918305BF
:1013F000C827E82FF0E0E658FA4F678589E70E9492
:10140000E2096C2F8DE30E94E2096C2F82E40E94B6
:10141000E209CF91089586E20E94DC090895CF93F6
:10142000DF93EC016C818CE10E94E2096D818DE11A
:101430000E94E2096E818EE10E94E2096F8180E2E2
:101440000E94E209688581E20E94E209698582E2E0
:101450000E94E2096A8583E20E94E2096B8584E2C8
:101460000E94E2096C8585E20E94E2096D858AE2AC
:101470000E94E2096E858EE60E94E2096F858FE682
:101480000E94E209688980E70E94E209698981E790
:101490000E94E2096A8982E70E94E209DF91CF9106
:1014A0000895CF92DF92EF92FF92CF93DF936B017B
:1014B0007C01C11488E3D8068CE9E8068CE1F806C3
:1014C00028F5C701B60120E836E948E950E00E9456
:1014D000592EE901689760E879E687E69FEF0E9458
:1014E000352E6C0D7D1D8E1D9F1DF2E0660F771F42
:1014F000881F991FFA95D1F721E732E040E050E0CC
:101500000E94592EF22EE32E80E421C0C701B601BD
:1015100020E03DE241E351E00E94592EE901689745
:1015200060E073ED8EEC9EEF0E94352E6C0D7D1DFC
:101530008E1D9F1D660F771F881F991F21E732E0C0
:1015400040E050E00E94592EF22EE32E80E66C2FF0
:101550006F71680F85E70E94E2096E2D86E70E9491
:10156000E2096F2D87E70E94E209DF91CF91FF909A
:10157000EF90DF90CF900895682F8DE60E94E209EA
:1015800008958F929F92AF92BF92CF92DF92EF9287
:10159000FF92CF93DF93D82F83E00E94DC098093E2
:1015A000750584E00E94DC098093740560E086E0A4
:1015B0000E94E20961E087E00E94E2096FE789E0AA
:1015C0000E94E20965E08AE00E94E20962E18BE0A4
:1015D0000E94E20965E18CE00E94E2096DEF8DE076
:1015E0000E94E20960E08EE00E94E209DD2319F02A
:1015F0008BE291E008C02091A10533E1239FC00157
:101600001124825C9E4F0E940F0A6CE880E30E94C6
:10161000E2096FE082E30E94E20962E483E30E9450
:10162000E2098091A20587FF02C064E101C06AE07F
:1016300084E30E94E2096AE285E30E94E2096DE226
:1016400086E30E94E20964ED87E30E94E20960E01C
:1016500088E30E94E20960E089E30E94E209D11177
:1016600009C0C0908305D0908405E0908505F09076
:10167000860507C0C5E9CC2EC1ECDC2EED2CCEEDE5
:10168000FC2ECAE38F2C9924AA24BB24682D8C2F0E
:101690000E94E209682D85E08C0F0E94E209FE2C71
:1016A000ED2CDC2CCC24CF5FCE3361F76FEF83E4DD
:1016B0000E94E2096FEF84E40E94E2096FEF85E483
:1016C0000E94E2096FEF86E40E94E209DD2311F037
:1016D00066E002C0609187058DE60E94E20960E045
:1016E00089E70E94E209609188058AE70E94E20981
:1016F00060E083E70E94E20960E084E70E94E2097B
:10170000D11109C060917F0570918005809181059C
:101710009091820504C060EC72E98DEE99E10E941F
:10172000510ADF91CF91FF90EF90DF90CF90BF9063
:10173000AF909F908F90089561E087E00E94E2094A
:1017400064E28EE70E94E20963E088E00E94E20919
:1017500060E088E00E94E20965E087E00E94E2091B
:1017600062E085E00E94E20983E00E94DC09809348
:10177000750584E00E94DC0980937405089583E078
:101780000E94DC098093750584E00E94DC09809347
:10179000740561E087E00E94E2096AE070E080E0A1
:1017A00090E00E9424290E949C0B00000895CF9293
:1017B000DF92FF920F931F93CF93DF931F92CDB7CA
:1017C000DEB7082F162F8EE399830E94E209F02ED0
:1017D000C02E9981D92E8C2D8F19811738F4F601DE
:1017E00061916F018FE70E94E209F5CF64E085E027
:1017F0000E94E20983E00E94DC098093750584E081
:101800000E94DC09809374050E9401296093700591
:1018100070937105809372059093730569E087E07A
:101820000E94E20981E0809377050F90DF91CF91CC
:101830001F910F91FF90DF90CF9008950F931F930A
:101840000E94D70B80917705813099F40E9401297D
:10185000009170051091710520917205309173050A
:10186000601B710B820B930B603A764881409105A7
:1018700048F380917705813031F46EE971E086EEAE
:1018800095E00E94ED2A1F910F9108950F931F93E9
:1018900080917705823021F41092770581E020C095
:1018A000809177058130D9F40E940129009170055B
:1018B000109171052091720530917305601B710BB9
:1018C000820B930B613A76488140910540F061E0CC
:1018D00087E00E94E2091092770582E001C080E073
:1018E0001F910F910895CF93DF93EC014AE050E0F0
:1018F0006D2F70E086EE95E00E94BB2B6EE286EEC7
:1019000095E00E94BF2ABE0184E0769567958A958E
:10191000E1F76F7077274AE050E086EE95E00E948D
:10192000BB2B6EE286EE95E00E94BF2ABE016F706F
:1019300077274AE050E086EE95E00E94BB2BDF91CE
:10194000CF910895D82FC0E0CD1780F4439A64E674
:1019500070E080E090E00E942429439864E670E003
:1019600080E090E00E942429CF5FEECF6CE271E02E
:1019700080E090E00E942429E6CF0F931F93CF933D
:10198000DF93EC01062F15E0115051F0CE010E94BB
:10199000B630081741F0602FCE010E94BE30F4CF60
:1019A00082E00E94A20CDF91CF911F910F910895C8
:1019B000A0E0B0E0EEEDFCE00C949C2E482E562EFC
:1019C000C0E0D0E0612C712CE12CF12C00E010E0A3
:1019D00041100CC06090D80586E4689E3001112447
:1019E00059E1E52EF12C0EEB15E01EC091E04912F5
:1019F0000FC06090D805E6E46E9E30011124FBE133
:101A00006F0E711C49E2E42EF12C0AE715E00CC0C0
:101A100082E0481209C028E1622E77247394EE24F4
:101A2000E394F12C07ED15E043018C0E9D1E1092FE
:101A30007905109278053401A62CA818B12CC301A1
:101A400001966C01AE14BF04A8F4A00EB11E511093
:101A500006C0C3010E94B630F501808305C0F501C0
:101A60006081C3010E94BD0CF50180810E94610666
:101A70003601E2CFC301511018C0C3010E94B63035
:101A8000B82EC6010E94B6302B2D30E0322F22270F
:101A9000282B80917805909179058217930779F426
:101AA000C0E0D0E05524539493CF3601609179057E
:101AB0000E94BD0C60917805C6010E94BD0CC05EFD
:101AC000DE4FC13E92E0D90708F482CF852DCDB715
:101AD000DEB7E0E10C94B82E61E082E00E94D80C01
:101AE000089560E082E00E94D80C8091D70585308F
:101AF00020F01092D7050E946C0D8091D70580933D
:101B0000D805089561E080E00E94D80C61E081E092
:101B10000E94D80C089560E080E00E94D80C8823D1
:101B200051F060E081E00E94D80C882321F0809180
:101B30007A05883349F00E94BF060E947A0681E048
:101B40000E94DF060E94820D0895882319F06AEA38
:101B500071E002C06EEA71E086EE95E00E94ED2A27
:101B60000895FF920F931F93CF93DF9369EC7BE06F
:101B700086EE95E00E94992A40917F05509180055C
:101B800060918105709182052AE030E086EE95E053
:101B90000E94C22B63EB7BE086EE95E00E94992ABF
:101BA000409183055091840560918505709186056B
:101BB00020E130E086EE95E00E94C22B6DE97BE0EB
:101BC00086EE95E00E94992A4AE050E060918705F0
:101BD00086EE95E00E94EA2B67E87BE086EE95E0D2
:101BE0000E94992A4AE050E06091880586EE95E0CF
:101BF0000E94EA2B61E77BE086EE95E00E94992A3D
:101C0000C9E8D5E0F12C8E0188818823A9F0FF2056
:101C100031F061EB71E086EE95E00E94BC2A2196DE
:101C20004AE050E0F801608186EE95E00E94B32B17
:101C3000F394F8E1FF12E7CF86EE95E00E94C72A01
:101C40006BE57BE086EE95E00E94992A4AE050E041
:101C50006091A10586EE95E00E94EA2B66E47BE0A8
:101C600086EE95E00E94992AE091A205E770F0E0E7
:101C7000EE0FFF1FEE57FC4F6081718186EE95E0FD
:101C80000E94ED2A61E37BE086EE95E00E94992AAE
:101C90008091A2058871883069F028F4811113C001
:101CA00068E27BE00CC0803141F0883161F46CE087
:101CB0007BE005C06CE17BE002C066E17BE086EE84
:101CC00095E00E94DB2A68EF7AE086EE95E00E94BC
:101CD000992A40917B0550917C0560917D0570911A
:101CE0007E052AE030E086EE95E00E94C22B6FED83
:101CF0007AE086EE95E00E94992A8091C305807172
:101D00000E94A50D66EC7AE086EE95E00E94992A85
:101D10008091C30580740E94A50D6DEA7AE086EE7D
:101D200095E00E94992A8091C30580720E94A50DBA
:101D300060E97AE086EE95E00E94992A8AE795E0CC
:101D40000E943708AB01BC012AE030E086EE95E046
:101D50000E94A42B6BE87AE086EE95E00E94992A17
:101D60008AE795E00E9437089B01AC0160E472E4C9
:101D70008FE090E00E94592EBA01A9012AE030E0DC
:101D800086EE95E00E94A42B68E87AE086EE95E066
:101D90000E94DB2ACDB7DEB7E5E00C94C32E8F920C
:101DA0009F92AF92BF92CF92DF92EF92FF928111FA
:101DB00007C06FE77AE086EE95E00E94DB2A2FC02D
:101DC00090E00E94740724E630E040E050E00E947A
:101DD000592ECA01B9012AE030E040E050E00E94EB
:101DE000592E49015A016B017C012AE030E0B5010E
:101DF000A40186EE95E00E94A42B6EE286EE95E0AB
:101E00000E94BF2A2AE030E0B701A60186EE95E0E5
:101E10000E94A42B63E786EE95E00E94FF2AFF90C4
:101E2000EF90DF90CF90BF90AF909F908F900895EC
:101E30001F93CF93DF9365E77AE086EE95E00E94EB
:101E4000992A8091A305813041F46CE57AE086EE11
:101E500095E00E94DB2A10E050C0823019F465E45E
:101E60007AE0F5CF843019F461E37AE0F0CF853081
:101E700091F766E27AE0EBCFC12FD0E0C930D1050F
:101E80000CF441C068E3610F86EE95E00E94BF2A22
:101E90006EE17AE086EE95E00E94992ABE016F5FBE
:101EA0007F4F4AE050E086EE95E00E94832B63E18D
:101EB0007AE086EE95E00E94992ACD55DA4FE981C5
:101EC000E03218F566E07AE086EE95E00E94992A05
:101ED0008981803130F06DE673E086EE95E00E94F6
:101EE000BC2A69816F7070E06F5F7F4F4AE050E0FD
:101EF00086EE95E00E948C2B1F5F80914C05181791
:101F000008F4BACF0FC061E3BECFEF70F0E0EE0F80
:101F1000FF1FEE56FC4F6081718186EE95E00E94B6
:101F2000ED2AEACF6BEE79E086EE95E00E94992AE1
:101F30008091BB050E94CF0E60ED79E086EE95E0C2
:101F40000E94992A8091BC050E94CF0E65EB79E032
:101F500086EE95E00E94992A8091BD050E94CF0EE1
:101F60006AE979E086EE95E00E94992A4091B305EE
:101F70005091B4056091B5057091B60541155105B4
:101F80006105710539F12AE030E086EE95E00E94A6
:101F9000C22B67E679E086EE95E00E94992A80914F
:101FA000B7050E949907AB01BC012AE030E086EE3C
:101FB00095E00E94C22B63E479E086EE95E00E94F2
:101FC000992A4AE050E06091B80586EE95E00E94BB
:101FD000EA2B06C06AE379E086EE95E00E94DB2AF0
:101FE0006DE179E086EE95E00E94992A6091B9054D
:101FF0007091BA054AE050E086EE95E00E94D42B3D
:1020000060E079E086EE95E00E94992A6091B20541
:10201000603450F470E06F5F7F4F4AE050E086EE2E
:1020200095E00E948C2B06C067EF78E086EE95E085
:102030000E94DB2A6AED78E086EE95E00E94992AFC
:102040008091B10580FF03C063EB71E002C067EBD4
:1020500071E086EE95E00E94ED2A6DEB78E086EE69
:1020600095E00E94992A8091B10582700E94A50D89
:102070006EE978E086EE95E00E94992A8091B1059C
:1020800084700E94A50D6FE778E086EE95E00E94CF
:10209000992A8091B10588700E94A50DDF91CF919A
:1020A0001F9108950F931F93CF93DF9320914905BC
:1020B0002F3FA9F56FEF75E086EE95E00E94992A13
:1020C00086E893E00E94730C6EED75E086EE95E075
:1020D0000E94992A80914A0590914B050E94730CA9
:1020E0006BEA75E086EE95E00E94DB2A68E875E011
:1020F00086EE95E00E94DB2A60E775E086EE95E0CB
:102100000E94DB2A6BE475E086EE95E00E94DB2AF4
:1021100086EE95E00E94C72A0E94180F68C012162A
:102120000CF065C0332727FD309580914C0590E079
:10213000821793070CF45BC066E375E086EE95E0CA
:102140000E94992A60914905772767FD70954AE0BA
:1021500050E086EE95E00E948C2B6BE075E086EEF9
:1021600095E00E94992A10E008E280914D05181729
:10217000D0F5C12FD0E0CC0FDD1FC25BDA4F288134
:1021800030E080914905992787FD909501972817A0
:10219000390739F56BEB71E086EE95E00E94BC2AB9
:1021A0004AE050E0602F86EE95E00E94B32B6FEB83
:1021B00071E086EE95E00E94BC2AE981EF70F0E0C4
:1021C000EE0FFF1FEE56FC4F6081718186EE95E0A9
:1021D0000E94BC2A63EC71E086EE95E00E94BC2A66
:1021E0000F5F1F5FC2CF86EE95E00E94C72ADF9186
:1021F000CF911F910F910895FF920F931F93CF934B
:10220000DF93C9E8D5E0F12C8E0188818823D1F1D4
:1022100065EC71E086EE95E00E94BC2A4AE050E051
:102220006F2D86EE95E00E94B32B62ED71E086EE95
:1022300095E00E94BC2A2196F801208130E0A0E1BF
:10224000B7E20E94132E9B01AC01A0918805B0E07B
:102250000E94222EAB01BC0180917F0590918005E8
:10226000A0918105B0918205480F591F6A1F7B1FFD
:102270002AE030E086EE95E00E94C22BF394F8E16C
:10228000FF12C2CFCDB7DEB7E5E00C94C32E10929B
:10229000E30485E6E4EEF4E0DF011D928A95E9F7B8
:1022A0000895CF93C82F8F3719F0883009F045C0B3
:1022B000E091E304EE23D9F1E150E093E304F0E090
:1022C000EC51FB4F10826DE070E086EE95E00E94CD
:1022D0005906C0E08091E304C81760F4EC2FF0E0E9
:1022E000EC51FB4F608170E086EE95E00E9459064C
:1022F000CF5FF0CF60E270E086EE95E00E94590675
:102300006DE070E086EE95E00E945906C0E0809195
:10231000E304C81778F5EC2FF0E0EC51FB4F608137
:1023200070E086EE95E00E945906CF5FF0CF67E03F
:1023300086EE95E00E94BF2A1DC08B3119F40E94E1
:1023400047111AC08D30C1F08A30B1F08091E3049A
:10235000843668F76C2F70E086EE95E00E9459068F
:10236000E091E30481E08E0F8093E304F0E0EC5110
:10237000FB4FC08380E001C081E0CF910895CF93EF
:10238000C82F0E9401296093CC047093CD048093E0
:10239000CE049093CF04C093E104CC2329F040E015
:1023A00051EE60E070E004C040E855E260E070E0AB
:1023B00086EE95E00E94492DCF9108959091D0042A
:1023C000492F4F7050E0BA016F5F7F4F292F30E0E7
:1023D000E4E035952795EA95E1F76217730759F020
:1023E000FA01EF52FB4F808381E0890F8F70907F5D
:1023F000892B8093D00408956EE770E086EE95E017
:102400000E9459060895A3E1B1E0E9E0F2E10C94DD
:102410009D2EE9E8F5E0712C8191882321F07394D9
:1024200028E17212F9CF66ED71E086EE95E00E9428
:10243000ED2A4AE050E0672D86EE95E00E94EA2BF7
:1024400080E00E94C10A0E949C0B8E010E5F1F4F0C
:10245000C12CD12C7601C39466246A945C2C0E9412
:10246000F5284B015C012091880530E0A0E1B7E23E
:102470000E94132E9B01AC01C701B6010E94352EAC
:1024800020917F0530918005409181055091820512
:10249000620F731F841F951F2091BF053091C005E7
:1024A0004091C1055091C2052617370748075907C3
:1024B00018F4F801608225C08C2D0E94F50961E0B6
:1024C00070E080E090E00E942429F80110820E94D0
:1024D000F528681979098A099B09643F71408105CB
:1024E000910540F40E940B0AF8019081981778F743
:1024F0008083EDCF50FE03C04298439A02C0429AB7
:1025000043982FEFC21AD20AE20AF20A0F5F1F4F56
:102510008FEFC816D104E104F10409F09FCFCE017A
:102520009395FC01D82E7FEF68EC2E2F281B2715E2
:1025300010F051E056C0DE01129651E02FEF41E05D
:102540003D91321710F0322F01C0452F5F5F5F3F82
:1025500011F0232FF5CF4193242F30E0A1E0B0E01C
:10256000AC0FBD1FA20FB31F5C93413079F0DE01A9
:10257000A20FB31F5C93423049F0AFEFBFEFAC0F37
:10258000BD1FA20FB31F6C934E3F78F6A2E0B0E0E0
:10259000AC0FBD1FA20FB31F7C934D3F30F6A3E0DD
:1025A000B0E0AC0FBD1FA20FB31F6C93BECF452F81
:1025B000242F30E0FC01E20FF31F6081AFEFB0E0A9
:1025C000AC0FBD1FA20FB31F2C91621748F44150EE
:1025D000DC01A40FB11D2C9120836C934111E8CF35
:1025E0005F5F571520F3372D369520E0231770F4E1
:1025F000DC01A20FB11D4C91522F530FFC01E50FCE
:10260000F11D50815C9340832E5FF0CFF9E8EF2EEF
:10261000F5E0FF2E8C01802F8D19871598F4F801B5
:10262000C1908F014AE050E06C2D86EE95E00E944B
:10263000B32B6CE286EE95E00E94BF2AF701C192AF
:102640007F01E9CF86EE95E00E94C72A81E0CD5E4A
:10265000DE4FEFE00C94B92E1F920F920FB60F923F
:1026600011241F932F933F934F935F936F937F9307
:102670008F939F93AF93BF93CF93DF93EF93FF938A
:10268000C0918600D0918700809187049091880442
:102690002091A904211155C09E01281B390B80915E
:1026A000C3059091C405A091C505B091C60585FDEF
:1026B00002C036952795253C49E03407B8F1409192
:1026C0000A0150E060E070E02CE1B695A79597957F
:1026D00087952A95D1F70097A105B10521F481E0EE
:1026E00090E0A0E0B0E084179507A607B707D8F4FC
:1026F00080910A018F3FB9F040E080910A014817AC
:1027000080F4842F90E0880F991FFC01E757FB4F5E
:1027100020813181FC01E55FFE4F318320834F5FD3
:10272000ECCF1092AA0410920A010BC02D3B82E05C
:10273000380720F080910A018031D8F08FEF809324
:102740000A01D0938804C0938704FF91EF91DF9131
:10275000CF91BF91AF919F918F917F916F915F9139
:102760004F913F912F911F910F900FBE0F901F908F
:10277000189510910A0181E0810F80930A01C90127
:102780000E942109E12FF0E0EE0FFF1FE757FB4FFA
:1027900091838083D6CF83E0809380008AE9809301
:1027A00081008091C30586FD05C080918100806411
:1027B000809381008FEF9FEF909389008093880032
:1027C00080916F00806280936F0008950E94710D68
:1027D0008091D805843011F41092D80508956F3097
:1027E00018F086958058089589E0689F802D1124FF
:1027F0000895A0E0B0E0EFEFF3E10C94A42EC82F11
:102800000E940129009138041091390420913A0462
:1028100030913B046B017C01C01AD10AE20AF30A31
:102820009701860149E8C41643E1D406E104F104A6
:1028300010F010923C046093380470933904809334
:102840003A0490933B042091A9048FEF820F8230C9
:10285000E8F5E0913C04EE2309F46EC1E13011F497
:1028600082E0D8C1E03178F581E08E0F80933C049E
:10287000F0E0E757FB4FC083803109F0D4C1EBE8AB
:10288000F4E0213029F4A181A695A695808108C0A5
:1028900080819181A92FA695A695A6959695879555
:1028A000A03148F4B0E090E0AA0FBB1FA55FBE4F77
:1028B00011969C938E931092AA04329684E0E93983
:1028C000F807F9F6B0C110923C04ADC1233009F00D
:1028D00023C1E0913C04E11118C0CF3009F011C1CF
:1028E0000E94F5280091B7041091B8042091B90412
:1028F0003091BA04601B710B820B930B623071052F
:102900008105910508F089C1FCC0E73148F481E0F8
:102910008E0F80933C04F0E0E857FB4FC083F1C07A
:10292000E73109F0ECC0C111EAC040E050E0ABE093
:10293000CA01B3E0880F991FBA95E1F7A49F9001EF
:10294000A59F300D1124F901E757FB4F6081E1810C
:102950007E2F777075956795FC01EE0FFF1FE55F81
:10296000FE4F71836083F901E657FB4FB081B69546
:10297000B695B695E181FE2FF295FF0FF07E6F2F91
:102980006B2BE695E695E6957E2F777075956795A6
:10299000FC01EE0FFF1FE35FFE4F71836083F901BF
:1029A000E557FB4FB081B295B695B695B370C1812E
:1029B000DC2FDD0FDD0F6D2F6B2BC295C695C695F5
:1029C000C370E281E170EE0FEE0F7E2F7C2B7595C8
:1029D0006795FC01EE0FFF1FE15FFE4F718360837F
:1029E000F901E357FB4FB081B695E181FE2FF795D2
:1029F000FF27F7956F2F6B2BE6957E2F77707595D8
:102A00006795FC01EE0FFF1FEF5EFE4F7183608341
:102A1000F901E257FB4FB081B295BF70E181FE2F03
:102A2000F295F07F6F2F6B2BE295EF707E2F777012
:102A300075956795FC01EE0FFF1FED5EFE4F7183EC
:102A40006083F901E157FB4FB081BB1FBB27BB1F60
:102A5000C181DC2FDD0F6D2F6B2BCC1FCC27CC1F42
:102A6000E281E370EE0F7E2F7C2B75956795FC015C
:102A7000EE0FFF1FEB5EFE4F71836083F901EF568F
:102A8000FB4FB081B695B695E181FE2FF295FF0F11
:102A9000FF0FF07C6F2F6B2BE695E6957E2F7770FE
:102AA00075956795FC01EE0FFF1FE95EFE4F718380
:102AB0006083F901EE56FB4F208122952695277001
:102AC0003181E32FEE0FEE0FEE0F6E2F622B732F7F
:102AD00072957695777075956795FC01EE0FFF1FDF
:102AE000E75EFE4F718360834F5F5F4F4230510559
:102AF00009F01ECF80919F0483FF1092AA041092C8
:102B00003C040E94F5286093B7047093B804809346
:102B1000B9049093BA0487C0243009F084C060914E
:102B20003C0461110BC0C83AB1F4109279051092BF
:102B3000780588EA0E94610681E06CC0613019F472
:102B4000C093370404C0623031F4C09336048C2F34
:102B50000E9461065AC0E09136042E2F30E0220F09
:102B6000331F462F50E0C9010296841795073CF0A9
:102B7000633268F7FA01EA57FB4FC083E8CF2D5F55
:102B80003F4F8C2F90E06091780570917905421746
:102B9000530749F4982F882786279727909379051C
:102BA0008093780532C06817790769F580913704FA
:102BB000813049F5E13118F080E180933604F090DE
:102BC0003604CAE8D4E000E010E00F15D0F4FE01AE
:102BD0003197808190E0982F88272881822B63E0AD
:102BE000969587956A95E1F70E942109F801EE0F05
:102BF000FF1FE55FFE4F918380830F5F1F4F22967B
:102C0000E4CF1092AA0410923C0480913C048823E3
:102C100051F08F5F80933C0406C080913C048F5F2D
:102C200080933C046ECFCDB7DEB7E8E00C94C02EA5
:102C3000E82FF0E0E254FA4FE185E03150F4F894E7
:102C4000F0E0EE0FFF1FE55FFE4F808191817894E9
:102C500008958EE08E0F8B3058F4F0E0E25FF109BA
:102C600024E62E9FC0012F9F900D11240C960895ED
:102C7000E03FF1F028F4E03161F0E13161F006C0AD
:102C8000ED3F81F0EE3F89F0E13F49F080E092E0D6
:102C9000089582E101C083E10E94432A089586E0FD
:102CA00090E008958AEF93E008958FEF93E0089500
:102CB00080E090E00895A2E2B0E0E1E6F6E10C9455
:102CC0009A2E9E012F5F3F4F80E1D9011D928A9578
:102CD000E9F764E072E086EE95E029A33AA30E944A
:102CE000ED2A0E94BF0B1D8A1E8A1F8A188E312C66
:102CF000212C00E0812C912C540170E4472E71EEC0
:102D0000572E7DE9672E78E1772EE0E5CE2EE3ECB5
:102D1000DE2EE12CF12C84EF91E0A0E0B0E08D8F6D
:102D20009E8FAF8FB8A380EC91EDA8E9BBE1898FAE
:102D30009A8FAB8FBC8F80E491EEADE9B8E1898BBF
:102D40009A8BAB8BBC8B86EE95E00E94012C892B75
:102D500009F4E1C086EE95E00E942E2C9C013327F9
:102D60002C32310509F442C0ACF42332310509F0AC
:102D7000ABC019821A821B821C821D821E821F8296
:102D8000188619861A861B861C861D861E861F8637
:102D9000188A60C02434310529F02335310509F43F
:102DA000B2C092C064E486EE95E00E94BF2A2AE099
:102DB00030E040E451EE6DE978E186EE95E00E9466
:102DC0004D2B6CE286EE95E00E94BF2A2AE030E0AF
:102DD00040EC51ED68E97BE186EE95E00E944D2BD9
:102DE0006CE286EE95E00E94FF2AADCF0F5F0430C3
:102DF00009F0A9CF29813A814B815C81A8EEB3E02B
:102E00000E94222E698B7A8B8B8B9C8B2D813E812D
:102E10004F8158850E94222E698F7A8F8B8F9C8FCD
:102E200029853A854B855C852D8F3E8F4F8F58A322
:102E30002D853E854F8558890E94222E6B017C018D
:102E400060323EE473078105910530F462E38CE162
:102E50000E94E20900E077CF603345E774078105FF
:102E6000910510F462E2F3CF60345CE975078105E7
:102E7000910510F466E2EBCF80E5C81683ECD80626
:102E8000E104F10410F462E1E2CF90E6C9169AEE93
:102E9000D906E104F10410F465E1D9CFA0E7CA1620
:102EA000A1E1DA06A1E0EA06F10410F461E0CFCF77
:102EB000B0EACB16B6E8DB06B1E0EB06F10410F49D
:102EC00063E0C5CF65E0C3CF10ED180F1A3008F0EE
:102ED0003ACFE1E0F0E0EC0FFD1F24E0029FE00DAF
:102EE000F11D11242081318142815381AAE0B0E09B
:102EF0000E94222E610F711D811D911D60837183BF
:102F00008283938320CF49885A886B887C88812C60
:102F1000912C540118CF81149104A104B10489F4B7
:102F2000C301B2010E94510A61E070E080E090E0CC
:102F30000E9424291D8A1E8A1F8A188E312C222461
:102F40002A948D8D9E8DAF8DB8A188169906AA06FC
:102F5000BB06D0F40E940B0A2D893E894F89588DFB
:102F6000280F311D411D511D2D8B3E8B4F8B588FCE
:102F7000381608F4382E821508F4282E3FEF831AED
:102F8000930AA30AB30A56C0C301B20128EE33E084
:102F900040E050E00E94592EBA01A9012AE030E039
:102FA00086EE95E00E94A42B6CE286EE95E00E94EE
:102FB000BF2A4AE050E0632D86EE95E00E94B32BD5
:102FC0006CE286EE95E00E94BF2A6D897E898F892A
:102FD000988DA50194010E94592EBA01A9012AE0F9
:102FE00030E086EE95E00E94A42B6CE286EE95E040
:102FF0000E94BF2A4AE050E0622D86EE95E00E94D2
:10300000B32B6CE286EE95E00E94FF2A4C0C5D1C0F
:103010006E1C7F1C898D9A8DAB8DBC8D841595059A
:10302000A605B70520F449885A886B887C88812CCE
:10303000912C540129893A894B895C89283E334077
:103040004105510509F07FCEA296E2E10C94B62E1F
:10305000ACE1B0E0EEE2F8E10C94A42E0E9401296C
:103060006B017C0181E00E94C10A14E703E019832F
:1030700061E0CE0101960E941E0C009377050E942C
:103080009C0B6AEF70E080E090E00E942429809120
:103090007705833089F486EE95E00E94012C892B18
:1030A00059F40E9401296C197D098E099F09603825
:1030B000734C894C9140D8F280917705833009F4A4
:1030C0004FC08FE70E94BA090E94CD0989838435D9
:1030D00011F083E05CC00E94CD0910924A058093F4
:1030E0004B050E94CD0920914A0530914B05280FD0
:1030F000311D30934B0520934A050E94CD098093E2
:103100004C050E94CD0980934D05813110F7F12CBB
:103110000F2D10E080914D0590E0880F991F081742
:10312000190740F40E94CD09F801E25BFA4F808351
:10313000F394EECF80E7898361E0CE0101960E948F
:103140001E0C83E0809377050E949C0B62E370E085
:1031500080E090E00E94242980917705833011F46B
:1031600082E015C08FE70E94BA090E94CD098983C9
:10317000803509F0AECF03EA15E00E94CD09F801D1
:1031800081938F01F5E00E3B1F07B9F781E06C9644
:10319000E8E00C94C02E80914905992787FD909511
:1031A000A92FB92FFC013196EB30F10508F066C06C
:1031B000EC5CFF4F0C94D12E62E778E086EE95E050
:1031C0000E94DB2A86E893E00E94730C6AE578E0AF
:1031D00086EE95E00E94DB2A65E378E086EE95E0D6
:1031E0000E94DB2A6BE078E086EE95E00E94DB2A05
:1031F0006AEE77E086EE95E00E94DB2A6DEB77E0E1
:1032000086EE95E00E94DB2A67E977E086EE95E09E
:103210000E94DB2A63E777E086EE95E00E94DB2AD6
:103220006CE477E086EE95E00E94DB2A86EE95E07E
:103230000E94C72A0E94B10D21C06FE277E01AC038
:103240006AE077E017C065EF76E014C066ED76E0DF
:1032500011C062E976E00EC06DE776E00BC068E66B
:1032600076E086EE95E00E94DB2A62E276E002C01C
:103270006CE076E086EE95E00E94DB2A6AE070E082
:1032800080E090E00E94242986EE95E00E94012CC7
:10329000892B29F086EE95E00E942E2CF5CF08951B
:1032A000ACE1B0E0E6E5F9E10C94A42E909149057B
:1032B0009F3F09F023C1482F50E0FA013A97EF36BB
:1032C000F10508F00FC1E15CFF4F0C94D12E61E1D4
:1032D00072E0A0C06DE172E086EE95E00E94ED2AFA
:1032E00085E789838BE1E3EAF5E0DE011296019040
:1032F0000D928A95E1F76CE1CE0101960E941E0CB9
:103300000E949C0B83E08093770568EC70E080E07E
:1033100090E00E94242980917705843009F0E2C072
:103320008FE70E94BA090E94CD098983853509F08B
:10333000D9C06DEE74E086EE95E00E94DB2A6FEC5A
:1033400074E086EE95E00E94DB2A61EB74E096C0A3
:1033500065E372E086EE95E00E94ED2A89E68983B6
:1033600061E0CE0101960E941E0C0E949C0B83E03E
:103370008093770568EC70E080E090E00E9424295B
:1033800080917705843009F0ADC08FE70E94BA09BB
:103390000E94CD0989838E010E5F1F4F7E014DE192
:1033A000E40EF11C0E94CD09F80181938F01EE1506
:1033B000FF05C1F78BE1FE013296A3EAB5E001906B
:1033C0000D928A95E1F78981893409F08BC063E910
:1033D00074E086EE95E00E94DB2A65E774E086EEF5
:1033E00095E00E94DB2A67E574E048C06FE472E074
:1033F00086EE95E00E94ED2A8EEF8093490572C01B
:1034000080528750805390914C05981708F066C001
:103410006EE572E086EE95E00E94ED2A63C084E1DD
:103420008093490560E274E029C085E180934905F5
:1034300069EE73E023C086E18093490562EB73E097
:103440001DC087E18093490568E673E017C088E1F5
:103450008093490567E573E011C089E180934905D0
:1034600063E473E00BC08AE1809349056EE273E088
:1034700005C08BE18093490566E073E086EE95E038
:103480000E94DB2A2FC06CEE72E086EE95E00E946F
:10349000DB2A8091B10591E01DC066ED72E086EEF9
:1034A00095E00E94DB2A8091B10592E013C061ECA7
:1034B00072E086EE95E00E94DB2A8091B10594E0EF
:1034C00009C066EA72E086EE95E00E94DB2A8091F0
:1034D000B10598E089278093B1058FEF8093490566
:1034E0000E94521086EE95E00E94012C892B09F46F
:1034F0005BC186EE95E00E942E2CF4CF0E94511104
:10350000882309F451C18091E304811104C08FEF35
:103510008093490541C140E050E060E070E084EEF6
:1035200094E00E94482F40914905042F112707FD80
:103530001095212F312FF8013197EB31F10508F06B
:103540001BC1E255FF4F0C94D12E552747FD5095D6
:1035500020914C0530E0241735070CF40DC18B0188
:103560009C01015011092109310900321105210581
:10357000310558F0C0904D05EFE4F5E0F12CD12C69
:10358000A8E2EA2E415051090FC0FA01ED55FA4F59
:1035900061506083D9C0DF0111972C9130E024176E
:1035A000350729F0F3943296FC10F5CFCBC00E2DE1
:1035B00010E020E030E0061717072807390741F42C
:1035C0002081DA01AD55BA4F11962C93DD24D394A6
:1035D000E394E8CF6F3F71058105910511F008F084
:1035E000CBC06093BB05B0C06F3F710581059105ED
:1035F00011F008F0C1C06093BC05A6C06F3F710513
:103600008105910511F008F0B7C06093BD059CC01D
:103610002091E40420622037E9F440E050E060E0CB
:1036200070E085EE94E00E94482F9B01AC01DC0124
:10363000CB010197A109B1090897A105B10508F0CF
:10364000AEC0A4EDB0E30E94222E6A5E7C4A8A4698
:10365000954E24C02636E9F440E050E060E070E08A
:1036600085EE94E00E94482F9B01AC01DC01CB0168
:103670000197A109B1090797A105B10508F08FC00D
:10368000A8EAB1E60E94222E645E7C438E46944EE8
:1036900005C0611571058105910579F08B019C01CB
:1036A0000054114E2D4938410138F0EF1F07FAEF51
:1036B0002F07F2E03F0708F05FC06093B3057093F7
:1036C000B4058093B5059093B6053EC06F3F710574
:1036D0008105910511F008F04FC06093B70534C023
:1036E0008B019C0101501109210931090F3F11057E
:1036F0002105310508F040C06093B80525C08B0155
:103700009C01045C1940210931090D344DE1140775
:103710002105310528F47093BA056093B90514C0EA
:10372000611571058105910521F48FEF8093B20534
:103730000BC06134710581059105F0F4615060930F
:10374000B20502C0DD20C1F08091E20481111AC0EF
:103750008091830590918405A0918505B09186059F
:103760000196A11DB11D8093830590938405A093BC
:103770008505B093860506C060E772E086EE95E0A9
:103780000E94ED2A0E9447118FEF809349056AE05D
:1037900086EE95E00E94FF2A0E94521005C061E06B
:1037A00070E080E090E07ACF6C96E8E00C94C02E58
:1037B0006AE572E086EE95E00E94DB2A62E472E040
:1037C00086EE95E00E94DB2A86EE95E00E94012CB1
:1037D000892B31F086EE95E00E942E2C0E94501924
:1037E0000E942818823029F0833051F46DE072E095
:1037F00002C064E272E086EE95E00E94DB2A089542
:103800008FEF809349051092E2040E94521080913C
:1038100049058E3F69F086EE95E00E94012C892BC8
:10382000B1F386EE95E00E942E2C0E945019EFCF46
:1038300008950F931F93109149051F3F09F0D2C0BF
:10384000893409F457C000F5883309F469C058F485
:10385000803309F477C008F061C08B3109F440C0AF
:103860008132B1F1B9C0813409F487C030F48933B1
:1038700009F466C0803461F1AFC0823409F48EC0AF
:10388000863409F448C0A8C0823609F487C078F4A9
:10389000883531F128F48235C1F18335E1F09CC0DF
:1038A0008A3509F494C0813609F467C095C082371F
:1038B00061F128F4863679F18936E1F08DC08837D8
:1038C00079F08A3709F483C0833709F085C003C0D3
:1038D00061E172E015C00E94820D6EE872E004C0E2
:1038E0000E948B0D68EA72E086EE95E00E94ED2A58
:1038F0008EEF70C00E947A060E94BF0667EC72E0ED
:1039000086EE95E00E94ED2A67C081E00E94DF0606
:1039100060EE72E0F5CF0E94FC105EC080535AC08A
:103920006AEF71E086EE95E00E94DB2A9091A20595
:1039300088E0890F8871977E892B8093A2051AC031
:1039400089E048C067EE71E086EE95E00E94DB2AD0
:103950008091C3059091C405A091C505B091C6059D
:1039600020E182278093C3059093C405A093C505E9
:10397000B093C605109349052FC061ED71E086EE46
:1039800095E00E94DB2A8091C3059091C405A09127
:10399000C505B091C60540E4842710C060EC71E015
:1039A00086EE95E00E94DB2A8091C3059091C405C4
:1039B000A091C505B091C60520E282278093C3057A
:1039C0009093C405A093C505B093C60502C00E949C
:1039D000D81B8FEF80934905809149058E3F09F0F0
:1039E000D4C0DDC00E945111882309F4D8C0809151
:1039F000E304811104C08FEF80934905C6C040E005
:103A000050E060E070E084EE94E00E94482F009166
:103A10004905112707FD1095212F312FF801319706
:103A2000E930F10508F0B4C0E753FF4F0C94D12EF4
:103A30008B019C010154114E2D4938410F37104F15
:103A40002A4F324008F0A4C060937F057093800530
:103A5000809381059093820577C06093830570936E
:103A60008405809385059093860581E08093E20428
:103A70006BC0683071058105910508F089C06093BD
:103A8000870562C08B019C01015011092109310990
:103A90000A3011052105310508F07AC060938805C8
:103AA00053C061EB71E084EE94E00E94823010E03C
:103AB000009799F00E945C30009779F0183130F44B
:103AC000E12FF0E0E658FA4F87871F5F61EB71E066
:103AD00080E090E00E948230EBCF1831A8F5E12F12
:103AE000F0E0E658FA4F17861F5FF7CF6530710593
:103AF0008105910508F04CC06093A10525C08B019C
:103B00009C010150110921093109063011052105D7
:103B10003105F0F52091A205287F262B2093A205E0
:103B200013C08B019C0101501109210931090115B4
:103B3000124C2140310560F560937B0570937C0544
:103B400080937D0590937E058091E204811113C0DE
:103B50008091830590918405A0918505B09186059B
:103B60000196A11DB11D8093830590938405A093B8
:103B70008505B09386050E9447118FEF8093490514
:103B80006AE086EE95E00E94FF2A0E94CB1807C0EB
:103B900060E772E086EE95E00E94ED2AECCF1F917F
:103BA0000F9108958FEF809349051092E2040E94CF
:103BB000CB18809149058E3F69F086EE95E00E9412
:103BC000012C892BB1F386EE95E00E942E2C0E94E9
:103BD000191CEFCF6AE070E080E090E00E94242999
:103BE00086EE95E00E94012C892B29F086EE95E067
:103BF0000E942E2CF5CF0895CF93C82F682F86EE04
:103C000095E00E945B2C90916E059C2790936E0529
:103C1000CF910895A1E0B0E0E0E1FEE10C94AA2E7E
:103C200099830E94FC1D9981892F0E94FC1D219679
:103C3000E2E00C94C62E1F93CF93DF93182FEB0175
:103C400010926E0565EB70E086EE95E00E945906D5
:103C500062E670E086EE95E00E945906812F0E9490
:103C6000FC1DCE010E940A1EDF91CF911F91089585
:103C700060916E0586EE95E00E945B2C0895A1E2AE
:103C8000B0E0E5E4FEE10C94A62E7B018A018C30C5
:103C900009F452C108F040C0863009F4BCC018F5E0
:103CA000833009F491C070F4813009F472C082301D
:103CB00009F049C26BE170E082E00E941B1E03EA3A
:103CC00015E078C0843009F487C0853009F03BC224
:103CD00060914D0570E0660F771F85E00E941B1E06
:103CE0000EE415E086C0893009F4A7C070F487306F
:103CF00009F49BC0883009F026C261E070E088E0DA
:103D00000E941B1E8091D80524C28A3009F4CAC0C3
:103D10008B3009F4F1C017C28A3609F474C1D8F4A3
:103D2000873609F439C138F4853609F40DC1863671
:103D300009F41EC108C2883609F436C1893609F073
:103D400002C261E070E089E60E941B1E0E947A06B2
:103D50000E94BF06F6C18D3609F4D3C138F48B3604
:103D600009F490C18C3609F499C1EDC18E3609F47D
:103D7000DDC1873C09F0E7C161E070E087EC0E949B
:103D80001B1E81E00E94FC1D0E94381E10926F05D0
:103D9000E4C169E270E081E00E941B1E0AE715E0C1
:103DA000F80181918F010E94FC1DF5E0033A1F0785
:103DB000B9F7D1C1F80181918F010E94FC1DF5E096
:103DC0000E3B1F07B9F7C7C161E070E083E00E94B6
:103DD0001B1E0E942818BDC161E070E084E00E94B3
:103DE0001B1E81E00E94FC1D0E94381E0E945B1673
:103DF000B4C180914D0590E0880F991F98012E5411
:103E000035402817390708F0A6C1F80181918F01C4
:103E10000E94FC1DEECF62E070E086E00E941B1E57
:103E200086E893E00E940A1E96C161E070E087E098
:103E30000E941B1E80914C058CC186E6898361E03F
:103E4000CE0101960E941E0C0E949C0B83E0809381
:103E5000770568EC70E080E090E00E942429809172
:103E600077058430D9F48FE70E94BA090E94CD0902
:103E70008983863469F460E270E089E00E941B1E49
:103E800010E20E94CD090E94FC1D1150D1F763C1C0
:103E900061E070E089E00E941B1E53C161E070E0A8
:103EA00089E054C169E170E08AE00E941B1E109213
:103EB000BE05209176058091C3059091C405A0911F
:103EC000C505B091C605222311F0806801C08F7727
:103ED0008093C3059093C405A093C505B093C60510
:103EE0000EEB15E0F80181918F010E94FC1DF5E0B9
:103EF000073D1F07B9F72FC161E270E08BE00E9418
:103F00001B1E8091AA048F3F39F08091AA0491E092
:103F1000980F9093AA0402C08091AA040E94FC1DED
:103F200010E0812F0E9418160E944C090E940A1E60
:103F30001F5F1031B1F70FC161E070E08CE00E94AB
:103F40001B1E8091D70505C161E070E085E60E94E7
:103F50001B1E89E2E816F10409F0FAC0D801EAE76D
:103F6000F5E08D91819385E0E33AF807D1F7E9C058
:103F700061E070E086E60E941B1EEBE1EE16F104A4
:103F800009F0E6C0D801E3EAF5E08D91819385E080
:103F9000EE3BF807D1F7D5C061E070E087E60E94FC
:103FA0001B1E0E94820DCDC061E070E088E60E9479
:103FB0001B1E85E789838BE1E3EAF5E0DE011296BB
:103FC00001900D928A95E1F76CE1CE0101960E9475
:103FD0001E0C0E949C0B83E08093770560E273E0E7
:103FE00080E090E00E94242980917705843009F0D8
:103FF000AFC08FE70E94BA090E94CD098983853539
:1040000009F0A6C09EC061E070E08AE60E941B1E17
:1040100089E6898361E0CE0101960E941E0C0E9410
:104020009C0B83E08093770560E273E080E090E092
:104030000E94242980917705843009F089C08FE798
:104040000E94BA090E94CD0989838E010E5F1F4F1D
:104050007E01EDE1EE0EF11C0E94CD09F801819385
:104060008F01EE15FF05C1F78BE1FE013296A3EA41
:10407000B5E001900D928A95E1F78981893409F0C4
:1040800067C05FC061E070E08BE60E941B1EF80114
:1040900080818093D8050E948B0D53C061E070E051
:1040A0008CE60E941B1EF0E2EF16F10461F487E635
:1040B000898380E2F801DE01129601900D928A95C3
:1040C000E1F761E203C087E4898361E0CE010196F4
:1040D0000E941E0C0E949C0B83E0809377056CE489
:1040E00074E080E090E00E9424298091770584307C
:1040F00079F58FE70E94BA090E94CD09873441F50E
:1041000020C061E070E08DE60E941B1E89E1E81688
:10411000F104F1F4D801EEEBF5E08D91819385E0A7
:10412000E73DF807D1F70E94CB130BC061E070E0C8
:104130008EE60E941B1EF80180818093D7050E94A5
:104140006C0D81E006C061E070E08AEC0E941B1EED
:1041500080E00E94FC1D0E94381EA196E6E00C94AF
:10416000C22EA0E0B0E0E7EBF0E20C94A42ECAEC83
:10417000D3E014E606E035E0F32E44E0E42E53E00D
:10418000D52E62E0C62E86EE95E00E94012C892B8A
:1041900009F49BC086EE95E00E942E2C282F809378
:1041A00035044091340450E04730510560F7FA017E
:1041B000EE52FF4F0C94D12E853B29F781E080937E
:1041C0003404E1CF823609F07DC0C0923404DBCFE5
:1041D0008093330480933204D0923404D4CF9C0172
:1041E0003327309331042093300490913204982780
:1041F00090933204E0923404C6CF382F22274091A6
:10420000300450913104242B352B3093310420930A
:10421000300490913204982790933204F092340441
:104220002536310508F4AFCF61E070E08CEC0E94D8
:104230001B1E81E00E94FC1D0E94381E43C020917D
:104240002E0430912F04F901E653FC4F80839091A6
:104250003204982790933204C901019690932F0459
:1042600080932E04209130043091310482179307FB
:1042700008F489CF0093340486CF809132048213EE
:104280000BC060912E0470912F044AEC53E0809192
:1042900033040E943F1E0DC062E070E08BEC0E9470
:1042A0001B1E809133040E94FC1D80916E050E94AC
:1042B000FC1DFE01812F11928A95E9F710922F04BF
:1042C00010922E04109234045ECFCDB7DEB7E8E032
:1042D0000C94C02E81E080936F0580916F05882338
:1042E00049F086EE95E00E94012C892BB1F30E94E3
:1042F000B120F3CF0895AAE2B0E0E1E8F1E20C9436
:10430000A22E0E94F5286B017C0181E00E94C10A67
:1043100086EE95E00E94012C892B29F086EE95E02F
:104320000E942E2CF5CF439811E072E6B72EE9E2F9
:10433000AE2E03E00E94F5286C197D098E099F09B5
:10434000693C710581059105D0F11123C1F10E94ED
:10435000F5286B017C01429A80ED97E00E94B60738
:10436000B982EAE7F5E0DE0112968A2D01900D92FE
:104370008A95E1F76AE2CE0101960E941E0C4298EE
:1043800080E090E00E94B607009377050E949C0BA6
:1043900062E370E080E090E00E942429809177053C
:1043A000843061F4009377058FE70E94BA090E9478
:1043B000CD0911E0823419F410E001C011E082E16E
:1043C0000E941A2A892B81F411E00EC0439A429A66
:1043D00086EE95E00E942E2C8D309105A9F05CF4BC
:1043E0000A9791F04398429886EE95E00E94012C3E
:1043F000892B61F79FCF8332910579F08234910543
:1044000089F70E946A21EECF62EB71E086EE95E0BB
:104410000E94DB2A0E94D21DE5CF0E945B16E2CFEC
:104420008F929F92AF92BF92CF92DF92EF92FF92C4
:104430001F93CF93DF9382E10E941A2A892B09F000
:1044400089C068EC70E080E090E00E94242980E060
:1044500090E00E94B6070E94F5284B015C016B01B9
:104460007C0180ECC80E82E1D81EE11CF11C0E9488
:10447000F5286C157D058E059F0530F482E10E94BC
:104480001A2A892BA1F364C082E10E941A2A892B7F
:1044900009F05EC080ED97E00E94B6070E94F52803
:1044A0006B017C01D0E0C1E088E4880E86E2981EB2
:1044B000A11CB11C11E082E10E941A2A892B21F56E
:1044C0008C149D04AE04BF0430F480ED97E00E948C
:1044D000B607D1E0F0CF0E94F5286C197D098E094E
:1044E0009F09693C71058105910528F30E94F52813
:1044F0006B017C01C12719F080ED97E002C080E0DC
:1045000090E00E94B607D7CF80E090E00E94B60707
:10451000DD23B9F08091D70590E0019665E070E069
:104520000E94452E8093D7050E946C0D0E94E613D1
:104530000E948B0D64EF71E080E090E00E942429DE
:1045400009C080E00E94DF060E9403120E94820DD3
:104550000E947B21DF91CF911F91FF90EF90DF9020
:10456000CF90BF90AF909F908F900895CF92DF92A1
:10457000EF92FF9280E00E941D080E94F40761E024
:1045800081E10E94AE2961E080E10E94AE2960E0F5
:1045900082E10E94AE2960E088E00E94AE2961E0DD
:1045A00088E00E94E7290E949F0740E052EC61E00A
:1045B00070E086EE95E00E94492D0E94E6130E946D
:1045C0008B0D0E94CB138FEF8093AA040E940908E1
:1045D00078940E94F5286B017C018091AA048F3F9A
:1045E00059F40E94F5286C197D098E099F09603DD8
:1045F00077408105910588F380ED97E00E94B6072A
:1046000061E082E10E94E729439A86EE95E00E94EC
:10461000012C892B29F086EE95E00E942E2CF5CFF7
:104620006DEF72E086EE95E00E94BC2A86E893E08A
:104630000E94730C64E173E086EE95E00E94BC2A50
:104640004AE050E068E070E086EE95E00E948C2B36
:1046500062E370E080E090E00E94242986EE95E01D
:104660000E94012C04970CF186EE95E00E942E2CFE
:1046700082349105D1F486EE95E00E942E2C8E3482
:10468000910599F486EE95E00E942E2C84349105D4
:1046900061F486EE95E00E942E2C819731F480E043
:1046A00090E00E94B6070E947B2140917B055091CB
:1046B0007C0560917D0570917E05DB01CA01019743
:1046C000A109B1090497A105B10568F44093A904B3
:1046D000433029F440EA56E861E070E004C040E06D
:1046E00052EC61E070E086EE95E00E94492D0E9458
:1046F0001022439880E090E00E94B6070E94CB13FE
:104700001092C9048091C30583FF11C080918F0569
:10471000882351F080919605882331F080919D0582
:10472000882311F087E001C085E08093C90480E010
:104730000E94C10A8091CA040E94F5090E949C0B44
:1047400010923F0410923E0410923D04F12C80918F
:10475000D8058F15B0F062E370E080E090E00E9431
:10476000242980ED97E00E94B60762E370E080E0C4
:1047700090E00E94242980E090E00E94B607F39424
:10478000E6CF8091A20584FF08C0982F987181E040
:10479000983109F080E00E94BF118FE00E941D084F
:1047A000FF90EF90DF90CF900895EF92FF920F93DC
:1047B0001F93CF93DF938C016EE770E086EE95E058
:1047C0000E945906E801F12CF0E2EF2E8E0188815B
:1047D0008D57823048F46DE770E086EE95E00E94D8
:1047E000590688818E2588832196F801608186EE9E
:1047F00095E00E945B2CF394F9E0FF12E7CF6EE79F
:1048000070E086EE95E00E945906CDB7DEB7E6E08F
:104810000C94C22EA9E0B0E0E0E1F4E20C94AA2EE0
:104820009091CB0491110EC09EEF99838A836B8384
:1048300050E0559547954C832D83198618861F8225
:104840001E822EC04091D004842F90E0B4E0959554
:104850008795BA95E1F7242F2F7030E082179307E0
:1048600019F18DEF89831B82FE01349650E0842F6D
:1048700090E0A4E095958795AA95E1F7242F2F70F5
:1048800030E08217930749F0DC01AF52BB4F8C91A7
:104890008193405F5F5F563051F74093D0045A8355
:1048A000CE0101960E94D5238091CB0490E0019621
:1048B00066E070E00E94452E8093CB042996E2E0EA
:1048C0000C94C62EA0E0B0E0E8E6F4E20C94A32E2F
:1048D0006C016EE770E086EE95E00E945906860155
:1048E000E12CF12CC0E0D0E030E2B32EF801608181
:1048F00083E8860F823078F46DE770E086EE95E00D
:104900000E945906F80160816B2570E086EE95E003
:104910000E94590604C086EE95E00E945B2CE114CB
:10492000F10459F0F80180819E01280F311DC90161
:10493000C92FDD27C80FD91FDD273FEFE31AF30A80
:1049400089E0E816F10459F028E0E216F10421F4B8
:104950008C2F8095F60180870F5F1F4FC7CFCDB793
:10496000DEB7E9E00C94BF2EA9E0B0E0EAEBF4E298
:104970000C94AA2EE82F362F8091CB0490E001965C
:1049800064E270E00E94452E8093CB0458E959837D
:1049900050E15A83813089F048F08230B9F0833099
:1049A000D9F48B8381EF8C833D8319C085E08B83A1
:1049B00081EF8C832F5F2D8312C08B8381EF8C83DB
:1049C00084E6489FA00111245D8309C084E08B83A5
:1049D00081EF8C83ED8303C00E94FC1104C0CE01E3
:1049E00001960E9462242996E2E00C94C62EA2E071
:1049F000B0E0EDEFF4E20C949F2E182F762E2A8370
:104A000049830E9401296B017C018091E10480901F
:104A1000CC049090CD04A090CE04B090CF042A8115
:104A200049818823C1F0D701C60188199909AA09CB
:104A3000BB094C015D0191EE89169EE29906A10425
:104A4000B10420F1241708F4422F202F672D812F65
:104A50000E94B42413C0D701C60188199909AA0974
:104A6000BB094C015D0191E3891695E79906A10404
:104A7000B10460F0672D812F0E940A24C092CC04FB
:104A8000D092CD04E092CE04F092CF042296EDE0D5
:104A90000C94BB2EA2E2B0E0E0E5F5E20C94A02E6F
:104AA0008CE00E94DC0981110DC06CE173E086EEA0
:104AB00095E00E94ED2A439A80E00E94C10A0E947C
:104AC0009C0B439886EE95E00E94012C892B01F106
:104AD00086EE95E00E942E2C9091A904992319F05E
:104AE0000E94F913EFCF40913E0450E09A012F5FEE
:104AF0003F4F2F71332760913F0470E0261737072F
:104B000009F3FA01E75BFB4F808320933E04DACF81
:104B100080917705843009F086C00E9401296115D3
:104B200071058105910549F06093BB047093BC0445
:104B30008093BD049093BE040CC081E090E0A0E09F
:104B4000B0E08093BB049093BC04A093BD04B093E9
:104B5000BE048091AD049091AE0481609093AE0448
:104B60008093AD0483E0809377058FE70E94BA09B4
:104B700009E614E00E94CD09F80181938F01F4E069
:104B800002371F07B9F72091720480916904982FAA
:104B9000922796FF3BC090E4922790937204982F3F
:104BA00098739833F1F410E0212F30E0809169047C
:104BB000877090E0821793074CF11F5F2091A20548
:104BC000812F90E0FC01E759FB4F24FF04C0808156
:104BD0000E94DE11E9CF608186EE95E00E945B2C99
:104BE000E3CF8F7399F480916A048093B604809127
:104BF0006B048093B40480916C048093B30480911F
:104C00006F0490E09093AC048093AB0480913D04DA
:104C1000813019F482E080933D0480913D0483301B
:104C200011F410923D040E9401296B017C018091D6
:104C3000AF049091B004A091B104B091B204009778
:104C4000A105B105C9F0A7019601281B390B4A0B34
:104C50005B0BDA01C901883B9B40A105B10560F0FF
:104C60000E940B0A8093B5041092AF041092B00416
:104C70001092B1041092B2048091BF049091C004CC
:104C8000A091C104B091C20446015701881A990A43
:104C9000AA0ABB0A8AE795E00E943708861697069B
:104CA000A806B90608F4A8C0C092BF04D092C004F8
:104CB000E092C104F092C2040E9457068091AA04B7
:104CC0008830A0F08091C3059091C405A091C505DE
:104CD000B091C6055CE1B695A795979587955A95CD
:104CE000D1F7892B8A2B8B2B09F0AAC18091AA04BA
:104CF0008F5F8093AA048091BB049091BC04A09123
:104D0000BD04B091BE040097A105B105F1F0C81A29
:104D1000D90AEA0AFB0A8AE795E00E9437086C156F
:104D20007D058E059F0508F012C18091C30584FDA5
:104D300004C080ED97E00E94B6071092BB04109269
:104D4000BC041092BD041092BE0490917204907C39
:104D50009093720450913E0480913F0420913D0451
:104D6000581709F411C1223009F00EC190589093E0
:104D70007204E091A205E770F0E0E658FC4F608114
:104D8000693008F0E9C0615040E04613E7C0809305
:104D90003F0487E3840F90917204892B80937204FF
:104DA0004093400483E080933D04429A80918705BC
:104DB0009091C904911135C10E94BC0A8091CA0426
:104DC0000E94F509E091A205E770F0E0E658FC4F7B
:104DD000608182E794E00E94D70BE091CA04EF5F04
:104DE000E093CA04E83109F428C1F0E0E658FA4F2C
:104DF0008785882309F421C10E94460C813069F51A
:104E00008091A205887149F18091AD049091AE0422
:104E1000880F991F9093AE048093AD0483E0809334
:104E200077050E949C0B0E9401296093AF04709348
:104E3000B0048093B1049093B204672B682B692B64
:104E400061F481E090E0A0E0B0E08093AF04909343
:104E5000B004A093B104B093B2048091A20584FF82
:104E60002BC08091BB049091BC04A091BD04B09173
:104E7000BE04892B8A2B8B2BF9F08091AD04909185
:104E8000AE048E7F0E946D09182F6091AB04809153
:104E9000B6040E94EF13482F612F8091B50449A3F7
:104EA0000E94EF130091D805282F49A16091B30407
:104EB0008091B4040E94F72442988091C704813005
:104EC000C1F018F08230B1F1C8C082E10E941A2A04
:104ED000892B09F0C2C081E08093C7040E94F528A5
:104EE0006093C3047093C4048093C5049093C60474
:104EF000B4C082E10E941A2A892B31F50E94F5285C
:104F0000C090C304D090C404E090C504F090C604DF
:104F10006C197D098E099F09693E734081059105D1
:104F200008F49BC082E08093C70480ED97E00E9464
:104F3000B60793C082E10E941A2A892B09F48DC01A
:104F400080E090E00E94B6071092C70486C080E01F
:104F500090E00E94B607F9CE68E016CF851709F4F5
:104F600016CF4F5F242F30E090E0F901EE58FB4F51
:104F7000DC01A75BBB4F7C917083F901E05CFB4FC8
:104F8000708301968F7101CF2430B1F420914004D9
:104F900081E494E0A3E7B4E0FC013E2F381B321714
:104FA00018F431913D93F9CF87E3820F9091720409
:104FB000892B80937204F6CE8091C704823051F41D
:104FC000916090937204439A8E010F5F1F4FF12CF2
:104FD000B80110C0439880913D04811103C081E065
:104FE00080933D0480913D04833071F784E0809389
:104FF0003D04EACF8F2D69A37AA30E941816F80109
:10500000819391938F01F39469A17AA1F0E1FF124A
:10501000F1CF8091A20543E754E087700E94BC085D
:10502000C4CE882309F4C8CE2091C80431E0320FE1
:105030003093C8042913C0CE0CC01092CA04DCCE31
:105040008091AA04883009F4439A89E08093AA04E5
:10505000D3CE1092C8048150AFCEA296ECE00C944F
:10506000BC2E8230E8F4E82FF0E0EE0FFF1FE7528D
:10507000FA4F71836083813041F0809169008C7FA9
:10508000842B80936900E89A089580916900440F09
:10509000551F440F551F837F842B80936900E99A25
:1050A00008951F920F920FB60F9211242F933F93E2
:1050B0004F935F936F937F938F939F93AF93BF9320
:1050C000EF93FF938091D9059091DA05892B29F010
:1050D000E091D905F091DA050995FF91EF91BF9123
:1050E000AF919F918F917F916F915F914F913F9180
:1050F0002F910F900FBE0F901F9018951F920F9237
:105100000FB60F9211242F933F934F935F936F939A
:105110007F938F939F93AF93BF93EF93FF93809170
:10512000DB059091DC05892B29F0E091DB05F091FE
:10513000DC050995FF91EF91BF91AF919F918F9100
:105140007F916F915F914F913F912F910F900FBE83
:105150000F901F9018951F920F920FB60F92112467
:105160002F933F938F939F93AF93BF938091DE05CF
:105170009091DF05A091E005B091E1053091DD054A
:1051800023E0230F2D3720F40196A11DB11D05C08A
:1051900026E8230F0296A11DB11D2093DD05809303
:1051A000DE059093DF05A093E005B093E1058091C3
:1051B000E2059091E305A091E405B091E505019623
:1051C000A11DB11D8093E2059093E305A093E40532
:1051D000B093E505BF91AF919F918F913F912F9132
:1051E0000F900FBE0F901F9018952FB7F8946091F5
:1051F000DE057091DF058091E0059091E1052FBFFC
:1052000008953FB7F8948091E2059091E305A0914D
:10521000E405B091E50526B5A89B05C02F3F19F020
:105220000196A11DB11D3FBF6627782F892F9A2FA8
:10523000620F711D811D911D42E0660F771F881F4F
:10524000991F4A95D1F70895CF92DF92EF92FF927E
:10525000CF93DF936B017C010E940129EB01C11404
:10526000D104E104F10479F00E9401296C1B7D0B4B
:10527000683E7340A0F381E0C81AD108E108F10844
:10528000C851DC4FECCFDF91CF91FF90EF90DF90D2
:10529000CF900895789484B5826084BD84B5816090
:1052A00084BD85B5826085BD85B5816085BDEEE62E
:1052B000F0E0808181608083E1E8F0E0108280810D
:1052C00082608083808181608083E0E8F0E080817B
:1052D00081608083E1EBF0E0808184608083E0EB9B
:1052E000F0E0808181608083EAE7F0E08081846083
:1052F00080838081826080838081816080838081DF
:10530000806880831092C1000895833081F028F472
:10531000813099F08230A1F008958630A9F087306D
:10532000B9F08430D1F4809180008F7D03C08091EA
:1053300080008F7780938000089584B58F7702C0B6
:1053400084B58F7D84BD08958091B0008F7703C0B0
:105350008091B0008F7D8093B0000895CF93DF934C
:1053600090E0FC01ED50F44F2491FC01E95FF34F14
:105370008491882349F190E0880F991FFC01E15D39
:10538000F34FA591B4918B5D934FFC01C591D491DE
:105390009FB7611108C0F8948C91209582238C935B
:1053A000888182230AC0623051F4F8948C91322FA4
:1053B000309583238C938881822B888304C0F89452
:1053C0008C91822B8C939FBFDF91CF910895A1E0A8
:1053D000B0E0EDEEF9E20C94A82E282F30E0F901B0
:1053E000E152F44F8491F901ED50F44F1491F90119
:1053F000E95FF34F04910023C9F0882321F069830A
:105400000E9485296981E02FF0E0EE0FFF1FEB5D20
:10541000F34FA591B4919FB7F8948C91611103C09B
:105420001095812301C0812B8C939FBF2196E4E0CE
:105430000C94C42ECF93DF93282F30E0F901E15272
:10544000F44F8491F901ED50F44FD491F901E95FE3
:10545000F34FC491CC2391F081110E948529EC2F48
:10546000F0E0EE0FFF1FE55EF34FA591B4912C9194
:105470002D2381E090E021F480E002C080E090E004
:10548000DF91CF9108958E3008F08E508770209173
:105490009D0190E4299F90011124822B80937C0030
:1054A00080917A00806480937A0080917A0086FDF2
:1054B000FCCF809178002091790090E0922B0895A4
:1054C000A0E0B0E0E6E6FAE20C94A42E6C017A01CA
:1054D000EB01E60EF71E00E010E0CE15DF0561F0EF
:1054E0006991D601ED91FC910190F081E02DC6010A
:1054F0000995080F191FF1CFC801CDB7DEB7E8E055
:105500000C94C02E6115710589F0DB010D9000200F
:10551000E9F7AD0141505109461B570BDC01ED91F4
:10552000FC910280F381E02D0995089580E090E0E0
:105530000895EF92FF920F931F93CF93DF938C0107
:10554000FB01C0E0D0E064917F018FEFE81AF80A18
:10555000662361F0D801ED91FC910190F081E02D7E
:10556000C8010995C80FD91FF701EDCFCE01CDB7FE
:10557000DEB7E6E00C94C22E0E94822A0895DC0178
:10558000ED91FC910190F081E02D099508950F9324
:105590001F93CF93DF93EC016DE00E94BF2A8C0133
:1055A0006AE0CE010E94BF2A800F911FDF91CF9148
:1055B0001F910F9108950F931F93CF93DF93EC01E9
:1055C0000E94992A8C01CE010E94C72A800F911F48
:1055D000DF91CF911F910F9108950F931F93CF9358
:1055E000DF93EC010E94822A8C01CE010E94C72A1F
:1055F000800F911FDF91CF911F910F9108950F930D
:105600001F93CF93DF93EC010E94BF2A8C01CE0140
:105610000E94C72A800F911FDF91CF911F910F9198
:105620000895A1E2B0E0E7E1FBE20C94A02E7C013A
:10563000C42EE52FCB01D22E19A221E02D1510F09A
:105640002AE0D22E8E010F5D1F4F8D2C912CA12CA4
:10565000B12C6C2D7E2FA50194010E94592E8C2D0A
:10566000D29E80191124015011098A3010F4805DF6
:1056700001C0895CF8018083211531054105510580
:1056800021F0C22EE32FCA01E4CFB801C7010E9466
:10569000822AA196ECE00C94BC2EA0E0B0E0E3E5F9
:1056A000FBE20C94A42EEC016A017B01211531056B
:1056B00041F4E881F9810190F081E02D642F099592
:1056C0001DC02A303105A9F477FF12C06DE20E9497
:1056D000BF2A8C0144275527BA014C195D096E0970
:1056E0007F092AE0CE010E94112B800F911F06C076
:1056F0002AE0B701A601CE010E94112BCDB7DEB77B
:10570000E8E00C94C02E9A01AB01662757FD609526
:10571000762F0E944D2B08950F931F93CF93DF9305
:10572000EC019A01AB01662757FD6095762F0E9428
:105730004D2B8C01CE010E94C72A800F911FDF9153
:10574000CF911F910F9108952115310549F4DC0186
:10575000ED91FC910190F081E02D642F0995089561
:105760000E94112B08959A01462F50E060E070E0EE
:105770000E94A42B08959A01AB0160E070E00E94A2
:10578000A42B08950F931F93CF93DF93EC010E94F6
:10579000A42B8C01CE010E94C72A800F911FDF919C
:1057A000CF911F910F9108950F931F93CF93DF9384
:1057B000EC019A01AB0160E070E00E94A42B8C0127
:1057C000CE010E94C72A800F911FDF91CF911F91B8
:1057D0000F9108950F931F93CF93DF93EC019A01DC
:1057E000462F50E060E070E00E94A42B8C01CE01B7
:1057F0000E94C72A800F911FDF91CF911F910F91B7
:105800000895FC0124853585F901E05CFF4F808116
:105810009181F901EE5BFF4F20813181821B930B57
:105820008F7399270895FC0184859585FC01E05CC0
:10583000FF4F40815181FC01EE5BFF4F20813181A0
:105840004217530741F00190F081E02DE80FF91F56
:10585000808190E008958FEF9FEF0895FC0184858B
:105860009585FC01E05CFF4F40815181FC01EE5BBE
:10587000FF4F208131814217530779F0A081B18118
:10588000A80FB91F8C91208131812F5F3F4F2F735B
:1058900033273183208390E008958FEF9FEF0895A1
:1058A000FC0181A1882329F0A489B5898C9186FF08
:1058B000FBCF11A20895CF93DF93FC012685378596
:1058C000D901A05CBF4F8D919C91119701968F7368
:1058D0009927E901CE5BDF4F4881598184179507ED
:1058E000D9F30D90BC91A02DA20FB31F6C93A68588
:1058F000B785A05CBF4F11969C938E93A689B789FC
:105900002C9181E090E0078C02C0880F991F0A94C7
:10591000E2F7282B2C9381E081A30488F589E02D00
:1059200080818064808381E090E0DF91CF91089551
:1059300008951F920F920FB60F9211242F933F9349
:105940004F938F939F93EF93FF938091C00082FDBD
:105950001CC04091C60080918C0690918D060196E6
:105960008F73992720918E0630918F0682179307A7
:1059700071F0E0918C06F0918D06E45BF94F408365
:1059800090938D0680938C0602C08091C600FF9193
:10599000EF919F918F914F913F912F910F900FBE5B
:1059A0000F901F90189586EE95E00E94012C892B90
:1059B00011F00E94982C08951F920F920FB60F922B
:1059C00011242F933F938F939F93EF93FF932091F5
:1059D00048063091490680914A0690914B06281757
:1059E000390731F48091C1008F7D8093C10014C0CC
:1059F000E0914A06F0914B06E85FF94F20818091D3
:105A00004A0690914B0601968F73992790934B0607
:105A100080934A062093C600FF91EF919F918F914A
:105A20003F912F910F900FBE0F901F901895A0E0FF
:105A3000B0E0EDE1FDE20C94A02EFC011382128295
:105A400088EE93E0A0E0B0E084839583A683B783DB
:105A50008CEB93E0918380837587648757874687B3
:105A6000318B208B138B028BF58AE48AD78AC68A06
:105A7000B18EA08E938E828E8F85848F8889858F3C
:105A80008989868F8A89878F8B8980A3ECE00C9423
:105A9000BC2ECF92DF92EF92FF92CF93DF93EC0177
:105AA0006A017B01411581EE580761057105F9F026
:105AB000EC89FD8981E090E008A002C0880F991F61
:105AC0000A94E2F7808360E079E08DE390E0A7013B
:105AD00096010E94592E21503109410951095695CC
:105AE000479537952795211580E1380798F0EC897F
:105AF000FD89108260E874E88EE190E0A7019601CC
:105B00000E94592E21503109410951095695479556
:105B100037952795E889F9893083EA89FB892083BD
:105B200019A2EE89FF89408181E090E09C010C8CF4
:105B300002C0220F331F0A94E2F7422B4083EE8902
:105B4000FF8940819C010D8C02C0220F331F0A94F3
:105B5000E2F7422B4083EE89FF8940819C010E8C45
:105B600002C0220F331F0A94E2F7422B4083EE89D2
:105B7000FF8920810F8C02C0880F991F0A94E2F7D9
:105B8000809582238083DF91CF91FF90EF90DF900B
:105B9000CF9008958F929F92AF92BF92CF92DF9253
:105BA000EF92FF920F931F9381E08F9385E08F9385
:105BB00087E08F9383E08F9384E08F93E6EC8E2EC3
:105BC000912CF2ECAF2EB12CA1ECCA2ED12CB0EC62
:105BD000EB2EF12C04EC10E025EC30E048E056E030
:105BE0006CE476E086EE95E00E94172D0F900F9002
:105BF0000F900F900F901F910F91FF90EF90DF90FB
:105C0000CF90BF90AF909F908F9008950E944A29A7
:105C10000E94B622C3EDDCE20E944A252097E1F300
:105C20000E94D32CF9CFA29FB001B39FC001A39FC4
:105C3000700D811D1124911DB29F700D811D1124C5
:105C4000911D08950E94132EA59F900DB49F900D55
:105C5000A49F800D911D11240895B7FF0C94222E4E
:105C60000E94222E821B930B0895DB018F939F933A
:105C70000E94222EBF91AF91A29F800D911DA39FE4
:105C8000900DB29F900D1124089597FB072E16F4E6
:105C9000009407D077FD09D00E94D72E07FC05D0CD
:105CA0003EF4909581959F4F0895709561957F4F33
:105CB0000895A1E21A2EAA1BBB1BFD010DC0AA1F4D
:105CC000BB1FEE1FFF1FA217B307E407F50720F065
:105CD000A21BB30BE40BF50B661F771F881F991FE0
:105CE0001A9469F760957095809590959B01AC0129
:105CF000BD01CF010895052E97FB1EF400940E946C
:105D0000922E57FD07D00E94592E07FC03D04EF467
:105D10000C94922E50954095309521953F4F4F4FC2
:105D20005F4F089590958095709561957F4F8F4F47
:105D30009F4F08952F923F924F925F926F927F9262
:105D40008F929F92AF92BF92CF92DF92EF92FF928B
:105D50000F931F93CF93DF93CDB7DEB7CA1BDB0B37
:105D60000FB6F894DEBF0FBECDBF09942A883988DC
:105D700048885F846E847D848C849B84AA84B984E3
:105D8000C884DF80EE80FD800C811B81AA81B981EF
:105D9000CE0FD11D0FB6F894DEBF0FBECDBFED0103
:105DA0000895EE0FFF1F0590F491E02D0994AA1BB2
:105DB000BB1B51E107C0AA1FBB1FA617B70710F0F6
:105DC000A61BB70B881F991F5A95A9F78095909528
:105DD000BC01CD0108958F929F92AF92BF92CF9256
:105DE000DF92EF92FF92CF93DF93EC01688179818C
:105DF0008A819B81611571058105910521F464E219
:105E000079ED8BE597E02DE133EF41E050E00E9422
:105E10007B2E49015A019B01AC01A7EAB1E40E9423
:105E2000222E6B017C01ACEEB4EFA50194010E941F
:105E3000302EC60ED71EE81EF91EF7FE06C081E002
:105E4000C81AD108E10880E8F80AC882D982EA8233
:105E5000FB82C701B6019F77DF91CF91FF90EF9052
:105E6000DF90CF90BF90AF909F908F9008950E9449
:105E7000EB2E089586E091E00E94EB2E089560934A
:105E8000060170930701809308019093090108951A
:105E90002F923F925F926F927F928F929F92AF92DA
:105EA000BF92CF92DF92EF92FF920F931F93CF9307
:105EB000DF938B01EA016115710521F0DB018C9301
:105EC00011969C93209739F09E012250310923327C
:105ED000310508F0D8C07C016701BFEFCB1ADB0A9F
:105EE0005601F7016080862D90E00E947A30892B60
:105EF00011F07601F1CFFDE26F120AC0570182E086
:105F0000A80EB11CD70111966C90772473940BC026
:105F1000BBE26B1207C05701E2E0AE0EB11CD70125
:105F200011966C90712CCE018F7E892B89F4B0E391
:105F30006B1237C0F50180818F7D8835D1F4618087
:105F4000F2E0AF0EB11C872D8260782EC0E1D0E068
:105F5000CA30D10551F1C031D10521F0C830D10589
:105F600099F409C0CC24CA94DC2CEC2CAFE0FA2EB6
:105F700022C0209769F7C8E0D0E0CC24CA94DC2C7A
:105F8000EC2CFFE1FF2E17C06FEF7FEFCB019E01DE
:105F9000442737FD4095542F0E94592E69017A01FC
:105FA0000AC02097A9F6CAE0D0E0E9E9CE2EDC2CA1
:105FB000EC2CE9E1FE2EF50160E020E030E0A901E3
:105FC0004E01AA2497FCA094BA2C1F0170ED572E05
:105FD000560CA9E0A51570F48FEB860D8A3118F4E4
:105FE00099EC592E06C08FE9860D8A3148F589EA69
:105FF000582E560C852D90E08C179D070CF56F3FA1
:10600000D9F0C216D306E406F50698F0C501B4012E
:106010000E94352E9B01AC01852D90E0A0E0B0E000
:10602000280F391F4A1F5B1F281739074A075B07CC
:1060300010F46FEF01C061E03196D1016C90C5CFD3
:106040000115110551F0662311F0319703C071FE5F
:1060500004C03297D801ED93FC9370FE07C05095B1
:106060004095309521953F4F4F4F5F4F67FF10C0D0
:1060700082E290E090939106809390066FEF7FEF1D
:106080008FEF9FEF07C060E070E080E090E002C01B
:10609000B901CA01DF91CF911F910F91FF90EF904D
:1060A000DF90CF90BF90AF909F908F907F906F9038
:1060B0005F903F902F900895FC0188279927E894DE
:1060C00021912032E9F3293010F02E30C8F32B3221
:1060D00041F02D3239F4689404C00E94AE30820F32
:1060E000911D219120532A30C0F31EF49095819583
:1060F0009F4F0895911150C0803219F089508550FA
:10610000D0F7089548EC53E00E9487300895FA01D3
:10611000A191B081009719F41097E1F0CD01DC0155
:10612000CD010D90002011F4C00113C0FB0121919D
:10613000222319F02015D9F7F3CFFB012191201567
:1061400019F41E92119606C02223C1F70D9000206B
:10615000A1F7D001FA01A193B08308957AE0979F47
:10616000902D879F802D910D11240895F999FECFD0
:1061700092BD81BDF89A992780B50895262FF99987
:10618000FECF1FBA92BD81BD20BD0FB6F894FA9A1A
:10619000F99A0FBE01960895992788270895F894D3
:0261A000FFCF2F
:1061A20000009206200001000000FF000200020031
:1061B20002000200020002000200020002000200CD
:1061C2000200020002000200020002802500000517
:1061D200400AA1204EA50020244EA52C2330C01237
:1061E20000001A400AA1204EA5001B1E27522C2394
:1061F200308025000005400AA1204EA50020244E33
:10620200A52C2330004B000006400AD0009D490017
:106212007B289D492C233000E1000005400A4501FE
:10622200D7DC03B81E0EBF00232E48E801008A40C7
:106232000A6001555502AD1E20000023C8015458C2
:106242002074696D656F75742100596573004E6F16
:10625200002C00386368004E2F41002C205B005D4B
:106262002028002900486F70206368616E6E656C9B
:10627200200020402000456E746572696E672061BF
:1062820064617074697665206368616E6E656C2006
:1062920073656C656374696F6E2C207069636B69DA
:1062A2006E673A007363616E6E6572206D6F64652E
:1062B200004E4F5420454E41424C45440053656EBA
:1062C20064696E672073657474696E677320746F96
:1062D2002052580A00526573657474696E672073A0
:1062E200657474696E6773206F6E2052580A00419C
:1062F200626F727465642065646974730A00696E02
:1063020076616C69642073656C656374696F6E0095
:106312000D0A496E76616C696420696E707574202D
:106322002D2064697363617264656421070053659B
:106332007474696E677320736176656420746F206C
:10634200454550524F4D0A00526576657274656438
:106352002073657474696E67732066726F6D204571
:106362004550524F4D0A004C6F616465642066616E
:1063720063746F72792064656661756C74730A0068
:106382004B657920616E64206368616E6E656C7323
:106392002072616E646F6D697A65640A004F706580
:1063A2006E4C52536E672054582073746172746934
:1063B2006E672000206F6E20485720006D6F647555
:1063C2006C65206C6F636B65643F00342B3400385E
:1063D20000382B340031320031322B340031360098
:1063E20050504D0052535349005344410053434CC3
:1063F20000525844005458440041494E004C424512
:1064020045500053504B54524D0053425553005384
:10641200554D44004C4C494E440000070B0C1011E2
:106422001500B7012B032F033103350338033D0356
:10643200B7014003440349034D0351035503590374
:106442005D0363036A036F0374038D028D028D0281
:106452008D02160A13223129000000005B2C602AEB
:08646200012C2E2C132C502CF0
:107E00000F92CDB7DEB7112484B714BE81FFF1D035
:107E100082E08093C00088E18093C10086E0809377
:107E2000C20080E18093C4008EE0CDD088249924E4
:107E3000CC24C394F5E0DF2EE1E1EE2E73E0F72EC3
:107E4000B6D0082F813479F4B2D08983C2D0898129
:107E5000823811F481E005C0813811F485E001C059
:107E600083E09ED09AC0823411F484E103C085344B
:107E700019F485E0B6D091C0853561F498D0082F0B
:107E800010E095D090E0982E8824802A912A880CC2
:107E9000991C82C0863521F484E0A3D080E0E1CF34
:107EA000843609F04CC083D082D0A82E80D0B82E62
:107EB00000E011E07CD0F80181938F01AE16D1F77C
:107EC00088D0FB2DF53489F4E0E0F1E00BC0F9999E
:107ED000FECF92BC81BC0894811C911C819180BD15
:107EE000FA9AF99AEA1598F358C08B2D863409F05E
:107EF00054C0F401F7BEE89507B600FCFDCFF401CD
:107F0000A0E0B1E02C9130E011968C91119790E0B7
:107F1000982F8827822B932B12960C01C7BEE895C9
:107F20001124329681E0A038B80761F7F401D7BE7A
:107F3000E89507B600FCFDCFE7BEE8952EC0843774
:107F4000F1F435D034D0182F32D0B82E42D0FB2DDA
:107F5000F63421F4F40105914F010CC0FB2DF534EA
:107F600049F4F999FECF92BC81BC0894811C911C04
:107F7000F89A00B5802F14D0115049F70EC08537FC
:107F800039F427D08EE10CD085E90AD08FE069CF93
:107F9000813511F488E017D01CD080E101D050CF9A
:107FA0009091C00095FFFCCF8093C600089580910A
:107FB000C00087FFFCCF8091C00084FD01C0A89560
:107FC0008091C6000895E0E6F0E098E19083808318
:107FD0000895EDDF803219F088E0F5DFFFCF84E10E
:107FE000DFCF1F93182FE3DF1150E9F7F2DF1F9166
:0E7FF0000895282E80E0E7DFEE27FF27099492
:027FFE0001057B
:0400000300007E007B
:00000001FF
